:100000000202863200000000000000320000000002
:10001000000000320000000000000032000000007C
:100020000000003200000000000000320000C0E0CC
:10003000741E1470FDD0E0002274C811451145D51E
:10004000E0F9D8F522C0E07419112E1470FBD0E04D
:1000500022D292C293A2E49294A2E59295A2E69251
:1000600096A2E79297D293C293A2E09294A2E192D1
:1000700095A2E29296A2E39297D293C293112E1187
:100080002E22C29280CDC292C2931145C297C296CF
:10009000D295D294D293C29311451145D293C29373
:1000A0001145D293C2931145C294D293C293114584
:1000B00074281182740E11827406118222748011C8
:1000C000822274C011822274021182114580EE7462
:1000D000011182114574801182220022D2B011DAFE
:1000E000D2B111DA7F0AD330B00C30B109DFF8C2D7
:1000F000B111DAC2B0C3920422C2B111DAD2B01186
:10010000DAD2B12292B111DA500C7F0A20B107DFA6
:10011000FBD2B0D38013D2B011DA7F0A20B007DF50
:10012000FBD2B1D38003C2B0C322D2B111DAD2B0B4
:1001300011DA7F0A20B005DFFBD38007A2B192D588
:10014000C2B0C3227E08333104400CDEF9312A40AC
:1001500006A2D5500211F9920422F874A6040000F8
:1001600000000000000070F500D8F022C3AE02E6E7
:1001700037F70809DEF922C3AE02E796F70809DE71
:10018000F922AE02760008DEFB22780C31822001D3
:1001900011C2D574082A14F8E630E706B2D57808FB
:1001A000510520010F74102A14F8E630E706B2D585
:1001B000781051057810790875F008EAA4FBE62656
:1001C000F6C0D0BA0104D0D0800BD0D0AE021E0849
:1001D000E633F6DEFA780CAE02E633F608DEFAAE67
:1001E00002780CE6970908DEFA19781040127908AF
:1001F000C3780CAE02E697F60908DEF97810190606
:100200007908DBBA22AE02D3E6F43400F608DEF851
:1002100022C0017910515ED001C00174102A14F877
:10022000E6C0E0780831827808760AE9240FF9E41C
:10023000F719C001318A780CD001E62430F7781024
:10024000AE02E44608DEFC70E8D0E020010730E7AB
:1002500004742D19F7A801D0017A10516722AE025B
:10026000E6F70809DEFA22E6F760040809DAF8E49E
:10027000F7227900E6080970FBE91422E66006120D
:1002800000510880F72275814D7520001200867597
:10029000339075340E753502753600C205B167B1FD
:1002A00073B1BA30070530B212C20720B20D740A1A
:1002B00012015A20B205D20712030630080530B3E6
:1002C00012C20820B30D740A12015A20B305D208D5
:1002D0001203A630090530B412C20920B40D740A05
:1002E00012015A20B405D209120446300A0530B56D
:1002F00012C20A20B50D740A12015A20B505D20A9D
:100300001205620202A3750819750900750A0075C5
:100310000B0085330C85340D85350E85360F780836
:10032000790C7A04316C850C33850D34850E358556
:100330000F36B1BAB1737464315A75F00030B2033C
:1003400075F0017400C395F0700302035002035767
:100350007490315A02035822750819750900750AFC
:1003600000750B0085330C85340D85350E85360FF1
:100370007808790C7A04316C850C33850D34850E40
:1003800035850F36B1BAB17374FA315A75F0003051
:10039000B20375F0017400C395F070030203A2026A
:1003A00003A502035822750819750900750A00751E
:1003B0000B0085330C85340D85350E85360F780896
:1003C000790C7A043177850C33850D34850E3585AB
:1003D0000F36B1BAB1737464315A75F00030B3039B
:1003E00075F0017400C395F070030203F00203F787
:1003F0007490315A0203F822750819750900750ABC
:1004000000750B0085330C85340D85350E85360F50
:100410007808790C7A043177850C33850D34850E94
:1004200035850F36B1BAB17374FA315A75F00030B0
:10043000B30375F0017400C395F070030204420227
:1004400004450203F822D2067508CC750929750AFD
:1004500000750B0085330C85340D85350E85360F00
:100460007808790C7A04316C850C33850D34850E4F
:1004700035850F3675F00030050375F0017401C342
:1004800095F0700302048A0204B6750858750902D3
:10049000750A00750B0085330C85340D85350E8586
:1004A000360F7808790C7A043177850C33850D3452
:1004B000850E35850F3675F00030050375F0017433
:1004C00001C395F070030204CC0204CEB1BAC2B7E6
:1004D000B17375F00030B40375F0017400C395F08A
:1004E00070030204E80204EB0204D2D2B7C206751C
:1004F00008CC750929750A00750B0085330C853405
:100500000D85350E85360F7808790C7A043177859C
:100510000C33850D34850E35850F3675F0003005AA
:100520000375F0017401C395F070030205310205F3
:100530005D750858750902750A00750B0085330C46
:1005400085340D85350E85360F7808790C7A04319F
:100550006C850C33850D34850E35850F36B1BAB1F7
:100560007322B205D14F2211DC74E43144E43144EA
:1005700011F922750819750900750A00750B0085B7
:1005800033108534118535128536137A04318A305B
:10059000D505781012020585103985113A85123B70
:1005A00085133C783908E6F537E539F53811DCE58F
:1005B000373144E538314411F92211CF853339857B
:1005C000343A85353B85363C75F00030060375F0CE
:1005D000017400C395F070030205DE02060A750877
:1005E000CC750929750A00750B0085330C85340D0F
:1005F00085350E85360F7808790C7A04316C850CB8
:1006000039850D3A850E3B850F3C78397A0479227D
:100610005111794578227A06120267793D7A03787A
:1006200045516777007A0378455172E8149AF87952
:10063000411202677700783D517C780BE8836006B1
:100640001200510880F602064B2E007841517C11B1
:10065000C711C2780BE88360061200510880F602C9
:100660000664200075F00030050375F0017401C3C5
:1006700095F0700302067A02068F11C711C2780B3B
:10068000E88360061200510880F602068F2D0022D2
:00000001FF
